:1000000027C036C035C034C033C032C031C030C064
:100010002FC02EC02DC0C1C02BC02AC029C028C0EF
:1000200027C000003A00370000003B003800010103
:100030000101010101010202020102040810204035
:10004000800402010000000000040302010000001F
:1000500011241FBECFE5D1E0DEBFCDBF20E0A0E67A
:10006000B0E001C01D92A936B207E1F7DCD0A2C111
:10007000C7CFE7E4F0E02491ECE3F0E09491E1E312
:10008000F0E0E491EE2361F12223B1F0223089F017
:1000900028F4213089F420B72F770DC0233029F0C0
:1000A000243051F42FB52F7D02C02FB52F772FBDEF
:1000B00003C020B72F7D20BFF0E0EE0FFF1FE85DEB
:1000C000FF4FA591B4912FB7F894811105C08C9181
:1000D000E92FE095E82302C0EC91E92BEC932FBFC8
:1000E00008953FB7F8948091650090916600A091C3
:1000F0006700B091680022B708B600FE05C02F3F28
:1001000019F00196A11DB11D3FBFBA2FA92F982F3D
:100110008827BC01CD01620F711D811D911D23E057
:1001200030E040E050E0C6D0B901CA0108958F9296
:100130009F92AF92BF92CF92DF92EF92FF92D1DF68
:100140004B015C0188EEC82E83E0D82EE12CF12C07
:10015000C8DFDC01CB0188199909AA09BB09883ECF
:100160009340A105B10558F021E0C21AD108E10879
:10017000F10888EE880E83E0981EA11CB11CC11402
:10018000D104E104F10421F7FF90EF90DF90CF90CC
:10019000BF90AF909F908F9008951F920F920FB6CF
:1001A0000F9211242F933F938F939F93AF93BF93FD
:1001B0008091610090916200A0916300B091640011
:1001C0003091600026E6230F2D3728F029EE230F0B
:1001D0000196A11DB11D2093600080936100909352
:1001E0006200A0936300B0936400809165009091D9
:1001F0006600A0916700B09168000196A11DB11D35
:100200008093650090936600A0936700B0936800A8
:10021000BF91AF919F918F913F912F910F900FBE02
:100220000F901F901895789480B7826080BF80B738
:10023000816080BF83B7826083BF83B7816083BFE3
:1002400089B7816089BF1EBC8EB582608EBD8EB5B8
:1002500081608EBD8FB581608FBD329A319A309AA0
:10026000379AECE3F0E02491E1E3F0E08491882315
:1002700099F090E0880F991FFC01EE5DFF4FA5916A
:10028000B491FC01E85DFF4F859194918FB7F8948C
:10029000EC91E22BEC938FBFC0E0D0E081E0E9DE8F
:1002A00046DF80E0E6DE43DF2097C1F3A9DEF6CF2C
:1002B00068940013E894A0E0B0E0E0E6F1E01DC02F
:1002C000EFEFE7F959016A015E23550FEE08FE2CA6
:1002D00087019B01AC019E23990F660B762FCB0102
:1002E0003BD0CDB7DEB7EAE024C02F923F924F92C9
:1002F0005F926F927F928F929F92AF92BF92CF92B6
:10030000DF92EF92FF920F931F93CF93DF93CDB7BE
:10031000DEB7CA1BDB0B0FB6F894DEBF0FBECDBF36
:1003200009942A88398848885F846E847D848C8407
:100330009B84AA84B984C884DF80EE80FD800C8110
:100340001B81AA81B981CE0FD11D0FB6F894DEBFF3
:100350000FBECDBFED010895DF93CF939F92A0E430
:100360009A2E0024D001E001F00116950795F7942C
:10037000E794D794C794B794A79448F41068A20F51
:10038000B31FC41FD51FE61FF71F081E191E220F1B
:10039000331F441F551F661F771F881F991F9A948C
:1003A00021F79D01AE01BF01C00111249F90CF91A3
:0803B000DF910895F894FFCFDE
:00000001FF
